:020000040000FA
:02000000282AAC
:02000800362C94
:1000100006110C280615000086101220280E12204A
:100020001C200800A8000F308605F0302805860443
:1000300006140000061008008316F03086048312B0
:10004000061100008614061406080610A8000614FF
:1000500006080610A81B232886108316F030860693
:1000600083120800861000000611000006100F30F1
:1000700029243030122005302924303012201A244F
:10008000303012201A24203012201A242830082060
:1000900008300820013008200630082008008316A8
:1000A000F030860483120615000086140614060834
:1000B0000610F039A800A80E061406080610F0393C
:1000C000A804A80E86108316F030860683121A2420
:1000D0002808080075208A110A12A70A0319A60A1F
:1000E000003E031908000A206A2826088A0027080B
:1000F0008200831203132008E1000130E20021088E
:1001000003198628E20D6210FF3E80286208E30092
:10011000E2098030200784006208800584136208A9
:10012000800508003A21E830F4000330F500F601BC
:10013000F70143212208F4002308F500F601F70136
:100140006F21F30CF20CF10CF00CF313F30CF20C26
:10015000F10CF00CF313F30CF20CF10CF00CF313A4
:100160007008E4007108E5003A212408F40025082D
:10017000F500F601F70143216408F4006508F50075
:10018000F601F7010330003E0319CD28F40DF50DFB
:10019000F60DF70D7410FF3EC4286F217008E800BB
:1001A0007108E9007208EA007308EB000A30F400F5
:1001B0000030F5006408F0006508F100F8217008CF
:1001C000E4007108E50000307102031DE9280330E6
:1001D00070020318EC280800610884006B08003CDA
:1001E000031DFC286A08003C031DFC286908003C2C
:1001F000031DFC286808003C0318372963088004A5
:10020000650803191329E601E70166086702031D63
:100210000B296508660203181329EC011522E60A6A
:100220000319E70A05296408EC0015226208800515
:10023000650803192B29E601E70166086702031D1B
:1002400023296508660203182B29EC011522E60A0A
:100250000319E70A1D296408EC0015220130E802A1
:10026000031CE902031CEA02031CEB02EE286208ED
:1002700080050800831203134030F0001F30F100A6
:10028000F201F3010800831203132230FC00F8018D
:10029000F901FA01FB01FC0303195F290310FB0CB0
:1002A000FA0CF90CF80CF30CF20CF10CF00C031C2A
:1002B0004B29FC0303195E2960214F2960210800A6
:1002C0007408F80775080318750FF90776080318FE
:1002D000760FFA0777080318770FFB0708008312D9
:1002E0000313FB01FA01F901F801E001730DF80DA8
:1002F0007408D421F30D0730FC00730DCE2174086F
:10030000731C8429D4218529E621F30DFC0B7D295A
:10031000720DCE217408731C8F29D4219029E621F7
:10032000F20D0730FC00720DCE217408721C9A2960
:10033000D4219B29E621F20DFC0B9329710DCE21CE
:100340007408721CA529D421A629E621F10D0730D5
:10035000FC00710DCE217408711CB029D421B12983
:10036000E621F10DFC0BA929700DCE217408711C3A
:10037000BB29D421BC29E621F00D0730FC00700D0B
:10038000CE217408701CC629D421C729E621F00D9E
:10039000FC0BBF297018CD2960210800F80DF90D5C
:1003A000FA0DFB0DE00D0800F8027508031C750F2F
:1003B000F9027608031C760FFA027708031C770F00
:1003C000FB020301031C0130E0020800F807750876
:1003D0000318750FF90776080318760FFA077708E0
:1003E0000318770FFB07030103180130E00708002B
:1003F00083120313F801F9011030FC00710DF80DA0
:10040000F90D7408F8027508031C750FF90203183A
:10041000102A7408F80775080318750FF9070310F8
:10042000F00DF10DFC0BFE29080083120313EC0301
:10043000EC036C08003C0318222AEC0300000000C7
:100440000000192A00000000000000000000080061
:1004500003138312850107309F0083163C3085000B
:100460008601803081000C1583120C110B3097002F
:1004700009309600C43095008B0183160C1083124E
:100480000C108F018E013130900086010630A000E3
:100490000330A100792032200C300820B123023033
:1004A000A900023008200230A6009830A7006A2078
:1004B000C03008206A2030242E24023008206A2010
:1004C000C03008206A2030242E24023008206A2000
:1004D000C03008206A2030242E24A90B512AD923A9
:1004E000013008203024831621309B001C141A0888
:1004F0008312B20083169B0A1C141A088312B300DD
:1005000083169B0A0301A52383169B0A0301A523D7
:10051000023008200230A600CE30A7006A20C0308A
:1005200008206A2042234B23B1018B170B17E02AC6
:100530002A3420344D346534743472346F346E345C
:1005400000346F346D3465342034493449342034F8
:100550002A34003420342034203420347634653476
:1005600072342E34003431342E3430343534203467
:100570002034203420340034203420346234793460
:1005800020346D342E347934003461346D34613468
:100590006D346F3474346F34203400344234653435
:1005A000613474343A3420342034543400346534A3
:1005B0006D3470346F343A342034203420340034B5
:1005C00008230514B830A2000130A3006430A40051
:1005D0000030A500922005102E080319F12A1323DC
:1005E000EC2A3208AF00AF0BF62A072B082385143C
:1005F000E030A2000630A3006430A4000030A50063
:10060000922085102E080319F32A1323022BE02AC7
:100610001730F1007030F000F5013308F400F821D4
:100620007008AE000800311D1B2B02303202031C83
:10063000392BB203222BB11D262B083032020318AE
:10064000392BB20A4223FF30B4003A2B311E2E2B35
:1006500029303302031C392BB303352BB11E3A2B3F
:10066000D23033020318392BB30A4B23FF30B500C5
:100670003A2B0124B101340303197C2335030319F8
:10068000912308003208BB003030BB0785300820BA
:100690003B080A2008003308B8005823C53008205A
:1006A00030303902031D562B2030B9007223080068
:1006B0003C3084005E235E235E2308000830B600D1
:1006C000B7010310B80DB70DF63037070318B700A0
:1006D0000318B80AB60B612B84033708800030304A
:1006E000800708000330B60038308400840A000810
:1006F0000A20B60B762B0800831621309B001C14B1
:100700001A088312320603190800831602309B0769
:100710001C149A0AA723831602309B028312320804
:10072000A52B831622309B001C141A088312330653
:1007300003190800831602309B071C149A0AA7238A
:10074000831602309B028312330883169A001C150D
:1007500055309D00AA309D009C149C18AD2B83122F
:1007600008000B30A2000230A300C830A400003003
:10077000A500922026249330A2000230A300C830A6
:10078000A4000030A500922026241030A2000330DF
:10079000A300C830A4000030A50092202624173002
:1007A000A2000430A3009030A4000130A5009220E4
:1007B00008001730A2000430A300C830A4000030A5
:1007C000A500922026241030A2000330A300C830D8
:1007D000A4000030A500922026249330A20002300D
:1007E000A300C830A4000030A500922026240B30BE
:1007F000A2000230A3009030A4000130A500922096
:1008000008001030A2000330A3004630A4000030DE
:10081000A500922008001730A2000430A300463043
:10082000A4000030A5009220080001241E302924D5
:100830000B2408002730AA001D2CAA0B1C2C080032
:100840000A30AB001A24AB0B222C08003230292CC2
:100850006430AC002024AC0B2A2C08000530312C6D
:100860000A30AD002824AD0B322C0800FD00030E29
:100870008301FE000A08FF008A010408ED008312CC
:1008800003130C1D5A2C0C11AE08031DAE03B40843
:10089000031DB403B508031DB503B0080319522C9A
:1008A000B0035A2C05083C393C3A03195A2CB100C4
:1008B0001930B0006D0884007F088A007E0E830026
:0608C000FD0E7D0E090093
:02400E00023F6F
:1042000043006F0070007900720069006700680069
:1042100074002000280043002900200032003000F4
:104220003100310020006200790020004D002E0096
:10423000590061006D0061006D006F0074006F0037
:06424000FF0004009600DF
:00000001FF
